:020000040000FA
:10000000001B0020F90200000103000003030000B0
:1000100005030000070300000903000000000000C2
:100020000000000000000000000000000B030000C2
:100030000D030000000000000F030000110300008A
:100040001303000081040000610800001303000096
:100050001303000013030000130300001303000048
:1000600013030000B5070000FD07000013030000A4
:100070001303000013030000130300001303000028
:100080001303000013030000130300001303000018
:100090001105000013030000130300001303000008
:1000A00013030000130300001303000013030000F8
:1000B0001303000013030000000000000000000014
:1000C00013030000130300001303000013030000D8
:1000D00013030000130300001303000013030000C8
:1000E00013030000130300001303000000000000CE
:1000F00000000000130300000000000013030000D4
:1001000000000000000000000000000000000000EF
:1001100000000000000000000000000000000000DF
:1001200000000000000000000000000000000000CF
:1001300000000000000000000000000000000000BF
:1001400000000000000000000000000000000000AF
:10015000000000000000000000000000000000009F
:10016000000000000000000000000000000000008F
:10017000000000000000000000000000000000007F
:10018000000000000000000000000000000000006F
:10019000000000000000000000000000000000005F
:1001A000000000000000000000000000000000004F
:1001B000000000000000000000000000000000003F
:1001C000000000000000000000000000000000002F
:1001D000000000000000000000000000000000001F
:1001E000000000000000000000000000000000000F
:1001F00000000000000000000000000000000000FF
:10020000DFF80CD000F0C6F800480047CD2700000A
:10021000001B002030B4044654E8000F0D4644E8AB
:100220000053002BF8D1156030BC704730B4044641
:1002300054E8000F40EA010544E80053002BF7D1D1
:10024000156030BC704730B4044654E8000F00EA33
:10025000010544E80053002BF7D1156030BC70470E
:1002600030B4044654E8000F80EA010544E8005326
:10027000002BF7D1156030BC704730B4044654E809
:10028000000F00EB010544E80053002BF7D1156087
:1002900030BC704730B4044654E8000FA0EB0105B1
:1002A00044E80053002BF7D1156030BC704770B4A0
:1002B00004464FF0000054E8006F0D68AE4207BFDF
:1002C00044E80023012044E800630E60002B1CBFBB
:1002D0000020F0E770BC704730B4044654E8000FCB
:1002E00088422CBF451A054644E80053002BF5D13F
:1002F000156030BC7047000006488047064800473C
:10030000FEE7FEE7FEE7FEE7FEE7FEE7FEE7FEE7C5
:10031000FEE7FEE785050000010200000048704787
:100320005C70000040EA01039B0703D009E008C9A4
:10033000121F08C0042AFAD203E011F8013B00F8AA
:10034000013B521EF9D27047D2B201E000F8012BF6
:10035000491EFBD270470022F6E710B513460A4645
:1003600004461946FFF7F0FF204610BD421C10F866
:10037000011B0029FBD1801A704730B504460020CC
:10038000034600E05B1C934203D2E05CCD5C401B63
:10039000F8D030BD064C074D06E0E06840F00103A0
:1003A00094E8070098471034AC42F6D3FFF72CFFCF
:1003B000F47000001471000030B58C1810F8012B97
:1003C00012F00F0301D110F8013B120906D110F809
:1003D000012B03E010F8015B01F8015B5B1EF9D112
:1003E00001E001F8013B521EFBD1A142E6D30020FF
:1003F00030BD00F01F02012191404009800000F152
:10040000E020C0F88012704700F01F0201219140E7
:100410004009800000F1E020C0F88012704700F031
:100420001F02012191404009800000F1E020C0F846
:100430008012704700F01F020121914040098000A6
:1004400000F1E020C0F88011704700F01F02012188
:1004500091404009800000F1E020C0F80011704791
:100460004907090E002806DA00F00F0000F1E0202D
:1004700080F8141D704700F1E02080F800147047E8
:1004800070B5204D28696C78401C2861687D10B1DA
:100490001D4802F099FB287803281AD11B48D0F890
:1004A0000C01B0B1012C04D0022C0AD01648123035
:1004B00023E02869032816D01348083002F084FB93
:1004C00011E02869022812D00F480D3002F07CFBA1
:1004D0000DE0032C0FD2012C05D0022C07D0BDE873
:1004E000704004F0A3BBBDE8704004F0CBBBBDE896
:1004F000704004F0DDBD04482830BDE8704002F0D3
:1005000063BB0000B407002038030A00001000405D
:1005100030B51B4C85B00025012080F31088D4F83D
:10052000D40038B3D4F8D00000EB800004EB800096
:1005300001798DF800108168C26803694069CDE9CE
:100540000330CDE90112D4F8D400401EC4F8D40021
:10055000D4F8D000401CC4F8D000D4F8D0000A2849
:1005600001D3C4F8D050002080F310882168684679
:100570008847D1E7002080F3108805B030BD000027
:10058000D007002030B54FF0805000228300D0F813
:100590003011C3F80C21C3F81021624B1A60624B72
:1005A0001B68624C2360604B1B1D1B68241D23606D
:1005B0005D4B08331B68241D23605B4B0C331B68A9
:1005C000241D2360584B10331B68241D2360564B99
:1005D00014331B68241D2360534B18331B68534C82
:1005E00020342360504B1C331B68241D23604E4B6A
:1005F00020331B68241D23604B4B24331B68241DB0
:100600002360494B28331B68241D2360464B2C3341
:100610001B68241D2360444B30331B68434C40341B
:100620002360414B34331B68241D23603E4B383319
:100630001B68241D23603C4B3C331B68241D236036
:10064000394B40331B68241D23600124082902D143
:10065000D0F8343113B1082904D006E0354B3449C1
:10066000196005E0D0F8343113B1082904D006E050
:10067000314BFB21196005E0D0F8343113B1082962
:1006800008D00EE090F858322C48016863F303015B
:10069000016002E0D0F834311BB929494FF40070F1
:1006A000086028480168C90702D06FF001010160A5
:1006B0002548016841F470010160BFF34F8FBFF31B
:1006C0006F8F4FF01021D1F80002002803DBD1F822
:1006D0000402002822DA1D4B1C601D480468002C0F
:1006E000FCD01224C1F800420568002DFCD0C1F8EE
:1006F000044201680029FCD01A6001680029FCD07E
:10070000BFF34F8F10487C380168124A01F4E06152
:1007100011430160BFF34F8F00BFFDE70F490E4843
:10072000086030BD380500400404001020C50040BA
:10073000488103008C56004018F50040E40E00404C
:10074000409602400004004088ED00E004E50140CE
:1007500000E401400400FA050090D003C40000202A
:10076000124A10B50021104B126809E053F82140DD
:10077000844203D10E4802F027FA13E0491CC9B2A3
:100780009142F3D3084A002112F1180201EB011340
:1007900002EB4303834201D1012010BD491CC9B2C1
:1007A0000629F3D3002010BD1C0A002034010020CC
:1007B000EC0003000E4800220178142905D2491CE0
:1007C000C9B201700A2901D302E00270022101E0DE
:1007D0006FF00101074803680B4403604368194444
:1007E0004160012141720448C0F8402102F006B97D
:1007F000060000204C0100200090004070B5144E0F
:100800004FF48030C6F808030025C6F84051114C5B
:10081000606810B9104802F0D7F9A570626801232A
:10082000656073640D480168001F00681430B1F5FD
:10083000804F04D2B0F5404F01D9637005E081428A
:1008400001D3012000E000206070BDE87040104737
:1008500000A000400C010020E500040044A5004079
:1008600001480068004700002800002002E008C896
:10087000121F08C1002AFAD170477047002001E01A
:1008800001C1121F002AFBD17047000072B605F0AB
:1008900097F900BF04F0EAFF0028FBD1104C0121BA
:1008A000208801EB00400FA105F0ECF8104800682B
:1008B000C00700D000BE2088022101EB00400DA13E
:1008C00005F0E0F8BFF34F8F0948E43801680D4A9E
:1008D00001F4E06111430160BFF34F8F00BFFDE7FA
:1008E00048010020466174616C206572726F72006D
:1008F000F0ED00E053797374656D20726573657473
:10090000000000000400FA050EB500210091CDE9B9
:1009100001106A4644F20100FFF7B8FF0EBD00F077
:1009200003B800F009B8000072B602480168491C1B
:10093000016070473000002003490868401E0860CD
:1009400000D162B6704700003000002070B5054647
:1009500008680C46411C04D002F072FE206802F0C8
:1009600030FE6068411C02D0002102F018FE2968A8
:10097000A069C1F82405607D227D29681043C1F873
:100980006C05D4E900122868C0F81425C0F80C15CD
:10099000207D012814D1A068411C02D0002102F062
:1009A000FEFDE068411C04D002F04AFEE06802F05F
:1009B00008FED4E902122868C0F80825C0F810150E
:1009C00070BD70B5054608680C46411C04D002F0A5
:1009D00041FE206802F0FFFD6068411C02D000214A
:1009E00002F0E6FD2968A069C1F82405607D217D3B
:1009F0002A680843C2F86C05D4E900122868C0F8D8
:100A00000C15C0F81425207D012814D1A068411CC4
:100A100002D0002102F0CCFDE068411C04D002F0BD
:100A200019FEE06802F0D7FDD4E902122868C0F888
:100A30000825C0F8101570BD084908B5085C00907D
:100A4000684602F0D3FDD0F810050099C84010F0B8
:100A5000010000D0012080F0010008BD3C6F0000C3
:100A60002DE9FC410646C0074FF000050ED0104F9F
:100A700000240122385D009500231146019502F003
:100A800031FD641C042CF4D300F01CF8B0070DD524
:100A9000074E0024361D0022305D032300951146C9
:100AA000019502F01FFD641C042CF4D3BDE8FC8109
:100AB000386F00000249085C012102F0D5BD00003A
:100AC000386F000010B500242046FFF7F3FF641CC8
:100AD000042CF9D310BD042801D2FFF7ADBF0020CC
:100AE000704710B50024FFF7BBFF204610BD000083
:100AF0002DE9F0470546861C90460F464FF0010948
:100B00000020FFF70CFF1B4C20683860D4E900017F
:100B1000401AA16804F21C47081A0EE00121384669
:100B200002F05AF801F004FE0146384602F054F88B
:100B3000D4E90001401AA168081A401C8642EDD889
:100B4000B8F1000F03D0052065F3891002E00620FC
:100B500065F39F50A2682168114004EB8101C860D1
:100B60002068304420600020FFF7DBFE4846BDE8E7
:100B7000F0870000D802002030B482680468531C5B
:100B80008360A154D0E901128A4202D330BC02F042
:100B9000B0BB30BC70470000034803C8814201D19C
:100BA0000120704700207047D802002010B50021B6
:100BB000024802F01CF880F3100010BDF40600207B
:100BC0002DE9F0411B4C1C4E4FF000052179607857
:100BD0004FF0030881434FF0010707D0257131889A
:100BE00008EB014015A104F04DFF01E000B12771B1
:100BF000E1782078814307D0E570318808EB014027
:100C000015A104F03FFF01E000B1E7706179A07821
:100C1000814307D06571318808EB014014A104F0CD
:100C200031FF01E000B1677104F020FE0028FBD124
:100C3000BDE8F08100000020480100205379737462
:100C4000656D2061646472657373206E6F742072C9
:100C50006563656976656400486F73742049442054
:100C60006E6F7420726563656976656400000000CC
:100C700044796E204B6579206E6F742072656365D0
:100C8000697665640000000002490A88028089785C
:100C900081707047846F00002DE9F0418AB02027F1
:100CA0000026099702F0E4FD054602F00BFE80469F
:100CB00002F08CFFC82002F017FF052002F04CFF65
:100CC000002002F0A5FD02F053FD00208DF8200069
:100CD00004460022012108A801F080FB30B1002069
:100CE00002F082FF641CE4B2642CF2D3C82000F04E
:100CF00017F901208DF820000146002208A801F014
:100D00006DFB08B31E480078F0B1002002F0B2FD80
:100D100000281DDD09AA69460020099702F042FD5E
:100D2000B0B19DF80000082812D11548DDF8011077
:100D30000C38C0F803100DF1010001F0B1FB0020E8
:100D400001F058FA012603E04FF4967000F0E8F83D
:100D50004FF4AF7000F0E4F802F038FF002002F02A
:100D600057FD002002F064FD284602F0BDFE40461B
:100D700002F0F2FE02F0FCFC0AB03046BDE8F08161
:100D8000BA000020002207E010F8013BFF2B01D041
:100D900000207047521CD2B28A42F5D3012070471E
:100DA000F0B50746204889B0154600780E4698B140
:100DB000012814D0022834D110221C4904A8FFF7BE
:100DC000B1FA1B490D2204A8FFF7ACFA0024164A19
:100DD0006846521C21460DE010221449F3E7102208
:100DE000124904A8FFF79EFA04A800F0D9F8EDE72D
:100DF000052C02D2135D035500E00155641CE4B2DA
:100E0000102CF5D302F058F804A802F067F86946F0
:100E1000084602F027F82B466A463146384601F06C
:100E20009FFB09B0F0BD0000A8000020876F000004
:100E30001C07002070B50C4605460D2910D800F09F
:100E40002BF808B1012070BD0648007840B901F0C8
:100E50008FF928B121462846BDE8704000F01CB843
:100E6000002070BDAE0000200149087070470000EE
:100E7000A800002001460D220148FFF753BA0000E8
:100E80001C07002003490268C1F80120007948715D
:100E900070470000A8000020F0B50746081D89B083
:100EA000C6B206208DF8100004AC0D46601CFFF79A
:100EB000EBFE2A463946201DFFF734FA174D2878F5
:100EC00008B1002000E00220FFF7CEFF701EC2B282
:100ED000611C601CFFF764FF01200090002301AA41
:100EE000314604A801F090FA18B99DF804000B28C7
:100EF00002D0002009B0F0BD01AC0322A01DA11D4D
:100F0000FFF74EFFA01D01F01FFB0028F2D028784C
:100F100010B9601CFFF7B6FF0120EBE7AE00002020
:100F200010B5044602F0BAFC6043400004D0034907
:100F3000BDE810408001084710BD0000A16F00000F
:100F4000F0B54E23B3FBF2F5022303704F23841850
:100F500004F8013C81B10123541E0BE003F00306A9
:100F60008E5DB6FBF5F705FB176605FB0366C654F9
:100F70005B1CDBB2A342F1DB01210DE04318445CB2
:100F800013F8013CE31ADBB2052B03D2C3F10503CE
:100F900023444354491CC9B29142EFD3F0BD000031
:100FA0000349D1F807200260C97A01717047000037
:100FB000AE00002041F6FF700078FF2801D001202C
:100FC00070470020704740F6817041F27E01095C55
:100FD000FF2905D00F20B0EB111F07D0080970477B
:100FE000401E00B20028F0DA0E20704701F00F001A
:100FF000704700000148407A704700004C01002013
:10100000FFFFFFFFFFFFFFFFFFFFFFFFFFFFFFFFF0
:10101000FFFFFFFFFFFFFFFFFFFFFFFFFFFFFFFFE0
:10102000FFFFFFFFFFFFFFFFFFFFFFFFFFFFFFFFD0
:10103000FFFFFFFFFFFFFFFFFFFFFFFFFFFFFFFFC0
:1020000010B588B000216FF0010002AAFF235354DD
:10201000491C09B20529FADB40F6817241F27E01C2
:10202000895CFF2917D00F20B0EB111F01D00C09DC
:1020300001E001F00F04214604A800F0D0F80522C9
:1020400002A905A8FEF799F910B1204608B010BD05
:102050004FF0FF30FAE7521E12B2002ADEDAF5E73F
:10206000F0B52F4D87B000262878012701ACB0B11C
:1020700003208DF80400601CFEF706FE0020FEF72A
:10208000F3FE0322611C601CFEF78AFE002303AAF4
:10209000042101A8009700F0B7F9A0B117E00220D1
:1020A0008DF804000521601C00F066F9012206216C
:1020B00001A800F093F950B1601CFEF7E3FE2F7009
:1020C000002007B0F0BD9DF80C00092802D02E704A
:1020D0000320F6E703AC0922601C611CFEF760FEDA
:1020E000601C00F031FAC0B19DF8100020B1012849
:1020F00005D0022800D12E709DF81000E1E7601D88
:1021000000F056F90D21074800F036F90548FEF7B2
:10211000B1FE012000F06EF8EDE72E700220D0E74E
:10212000AE000020290700203EB5104C0020207092
:10213000FEF740FF98B94FF4805090F87E00FF28DA
:102140000DD0FEF740FF01460E2808D2684600F089
:1021500046F80098C4F8030001A800F029F9BDE88A
:102160003E400248C01C00F09BB90000AE000020B9
:1021700010B58AB004208DF80400012001460090BB
:10218000002306AA01A800F03FF930BB9DF8180013
:102190000A2822D10DF11900FEF774FE05208DF8F2
:1021A000040001AC601CFEF76FFD0D21201D00F046
:1021B000E3F8201DFEF75EFE0120FEF755FE10221B
:1021C000611C601CFEF7ECFD0122112101A800F04A
:1021D00005F910B101200AB010BD0020FBE701EBAA
:1021E000C10101F580510A6802604A684260097ABB
:1021F000017270472DE9FE4300265E4FB04634461B
:1022000000285ED00025E94629466846FFF7E7FF2B
:1022100058490422C91C6846FEF7AFF838B9554939
:102220000522C91D09F10400FEF7A7F880B16D1C55
:10223000EDB20E2DE8D3002529466846FFF7CFFF03
:102240004C490422C91C6846FEF797F810B10CE00F
:102250002C4632E0052109F10400FEF793FD20B180
:10226000D7F807000190F87A13E06D1CEDB20E2D3F
:10227000E2D3002529466846FFF7B1FF09216846E9
:10228000FEF780FD48B157F8030F00907868019081
:10229000387A8DF808002C4631E06D1CEDB20E2D19
:1022A000E8D3B8F1000F07D004EBC4006946092257
:1022B00000F5805003F0E8FD3EB3FEF77BFE28B347
:1022C00056E0002421466846FFF789FF2949042289
:1022D000C91C6846FEF751F80028EED0641CE4B231
:1022E0000E2CEFD3002421466846FFF778FF042127
:1022F0006846FEF747FD20B1D7F80300009001269D
:10230000D2E7641CE4B20E2CEDD331E0FEF75BFEA5
:10231000A0422DD00E2C2BD04FF48051002040F63F
:1023200081720F2591F87E10531C04E041F27E016A
:102330009042095C0DD0CE43360706D0B5EB111F95
:102340000AD164F31F11C9B20AE001F0F001214380
:1023500006E044F0E00103E0401C00B29842E5DBF7
:1023600041F27E02104403F06DFD0120BDE8FE83C2
:102370000020FBE7AE000020F0B50B4B0025C3F8B2
:10238000005101241C602A46084E09E0D3F8007170
:10239000002FFBD037688754C3F80051521CD2B2CB
:1023A0008A42F3D35C60F0BD00D0004008D5004005
:1023B00003490268C1F807200079C872704700001D
:1023C000AE00002010B5044601F0AAF900E030BFCD
:1023D00001F05EFAB0EB440FF9D310BD10B5094C13
:1023E000134600226270A2700A460146184601F0A8
:1023F0004FF908B910BD30BF60780028FBD0A07835
:1024000010BD0000AE0000202DE9FC4780460A20E8
:102410000A9D009016460F46284601F0E5FB012470
:1024200001F098F901F0B4FA0028FBD101F02EFA7E
:1024300081461E2001F070FB01F09AF92A463946C8
:102440004046FFF7CBFFE0B10224284601F0CCFB69
:1024500007208DF804000A20FFF7B4FF2A46012167
:1024600001A8FFF7BBFF60B1284601F003FA40B1B5
:10247000202000906A463146284601F093F900B1C9
:10248000002401F067F900BF01F082FA0028FBD1B7
:10249000484601F041FB01F06BF92046BDE8FC879E
:1024A0002DE9FF41054601F073FA264C0646EDB3CF
:1024B00028786978EA7800EB0120A978090401EB13
:1024C0000261471801F082FB204601F09BFA50B1EF
:1024D0000021084601F082FA28B1384601F0A2FA3C
:1024E00008B1012402E0012407E037B12146084683
:1024F00001F074FA08B1012700E00027641CE4B27F
:10250000082CF2D301F0A8F90446C2B22946684665
:10251000FEF716FD87B12146684601F093FA58B1DF
:102520000120002E05D001F023F900E007E030B1D2
:10253000012004B0BDE8F0810020002EF9D0002079
:10254000F7E700000405070B10B503220349FDF768
:1025500014FF08B1002010BD012010BD846F0000E1
:1025600070B5002409E000BF11F8015B12F8016B9F
:102570007540641C00F8015BE4B29C42F4D370BD6A
:102580000278521C027002788A4201D30021017045
:10259000704700002DE9FC5F0E008346DDE90C4723
:1025A000C6F1000098469246814600D408460125AF
:1025B00003E000BF90FBFAF06D1C5045FADAA84525
:1025C00000D9454624B1002E01DB780700D5641EF2
:1025D000B80702D5B8F1000F0AD0F80708D13CB10E
:1025E000A54205D220215846641EFEF7C5FAF6E73B
:1025F000002E02DA4E462D2102E0780703D52B216A
:102600005846FEF7B9FA07F0030002280BD1B8F1DB
:10261000000F08D13CB1A54205D230215846641EB6
:10262000FEF7AAFAF6E7CDE900474346524631469F
:10263000584604F027FCBDE8FC9F000070B50D462D
:10264000044600684FF4887103F050FE4FF4907117
:10265000206803F04BFE4FF49271206803F046FEB1
:102660004FF4A271206803F041FE20681249C0F8BF
:10267000041320686907000B40B2090E002806DA2F
:1026800000F00F0000F1E02080F8141D03E000F1DD
:10269000E02080F8001420680121000B40B200F017
:1026A0001F0291404009800000F1E020C0F8801234
:1026B000C0F8001170BD00001003020002460020A7
:1026C0001268930702D0530702D47047500714D5FD
:1026D00002F00300012802D002280CD105E0C2F369
:1026E00083100B68801C184404E00223086803EB85
:1026F00092521044086001207047086800EB925322
:10270000C2F38910401CEEE70022027002214254FD
:10271000491CC9B20829FAD370470022027004216B
:10272000817003214254491CC9B20829FAD3704769
:102730002DE9FF410026234800F04BFA2148001FF5
:10274000074600F046FA204C60680090A56800E05B
:1027500000986946284004EB80000C30FFF7AEFF7C
:102760000028F5D101AA009901EA050304EB8303CF
:10277000491CDB6842F82030401C00910228F2D34B
:10278000019800F0030001280BD0022810D1019815
:10279000032101EB90500099BDF80A6001EB900015
:1027A00005E00198BDF80A60C0F38310084400906A
:1027B000384600F00BFA08B10098606004B030466B
:1027C000BDE8F081F0060020D802002000210220A0
:1027D000FEF787F94FF40041002003F0ADF908B18E
:1027E000FEF792F803F034F836480321008801EB35
:1027F000004035A103F046F903F038F80028FBD17A
:10280000012000F0CDF810B90020FEF77DF800F0AF
:10281000BFF8002001F078F828B901F023F800F59E
:102820000340FEF771F8962001F05EF9002001F0F8
:1028300043F928B901F016F800F50340FEF764F8F3
:102840004FF4FC7001F078F928B901F00BF800F5AD
:102850000340FEF759F8002001F05EF928B901F0B5
:1028600001F800F50340FEF74FF8FFF7C9FB00231E
:102870001C4910F1020F05D00122B0F1FF3F04D036
:102880000A7003E00B704B7001E00B704A70FFF7A9
:102890004BFC00F06DFF28B900F0E4FF00F50340A9
:1028A000FEF732F80120FEF716F908B104F090F8AF
:1028B0000020FEF710F908B104F018F8FEF780F9CF
:1028C000F0E70000480100204465736B746F7020CE
:1028D000656D756C61746F72206578616D706C6583
:1028E00000000000000000202DE9F047C7880446E2
:1028F000181D16468946B0FBF7F1B0FBF7F207FB4F
:1029000012009A193A44D21CB2FBF7F2DDF820A06B
:1029100001E02468491E0029FBD13D1A8846B542D2
:1029200016D818E0BAF1000F05D0211809EB0800FD
:102930002A46091D04E0204409EB08012A46001D2F
:10294000FDF7F0FC00202468761BA844B74201D9AB
:10295000354600E03D46002EE4D1BDE8F08700009A
:1029600030B5024659B103F013F90021074C09E0D4
:1029700004EB810315685B88AB4202D11160002033
:1029800030BD491C8142F3D3052030BD3801002001
:1029900002480121C16001607047000000900040C2
:1029A000134A0021116051605172117211490122C4
:1029B0004A60CA60931EC1F808331304C1F8043397
:1029C000C1F800220C4A042111600B49303110B1CA
:1029D0004FF4FA5001E04FF47A6008604FF0E021C4
:1029E0004FF40070C1F88002C1F800010120704767
:1029F0004C010020009000401095004070470000FE
:102A00000B4910B54A7A8AB1022202708A88427054
:102A10000B88C2F3032242EA031484701A09C270BD
:102A20000020086048604872012010BD002010BDE1
:102A30004C0100202DE9F0415C4903780446D1E9BE
:102A400003020025082B77D2DFE803F0042B487738
:102A5000726E8795217C914208D238B100EB8101DA
:102A60008A6C521C8A640168491C0160A17B2E4655
:102A700061F307062189677B61F31F4661896068FE
:102A800061F30F05217B61F31745E17B61F31F655E
:102A900001F0DAFC2A4631463846BDE8F04100F044
:102AA0004FBE4869407D10B9414800F08DF82F466F
:102AB000218965F3070761F31F476189267B61F36D
:102AC0000F05617B606861F31F6501F0BDFC2A465C
:102AD00039463046BDE8F04100F028BE217B9142E6
:102AE00008D238B100EB81018A6C521C8A640168FB
:102AF000491C0160A07A217A60F3070561F30F2574
:102B0000E17A667A676861F3174538B11FB92848DA
:102B1000263000F059F8384601F096FC2946304638
:102B2000BDE8F04100F0EFBEBDE8F04100F01EBE90
:102B300000F034FFBDE8F08131E01E484168491CD7
:102B4000416001780029F5D0816811B1491E81608A
:102B5000F0E7BDE8F04100F0FDBDA379934208D253
:102B600038B100EB830293685B1C93604268521C8F
:102B700042608A680CE0A379934208D238B100EB36
:102B8000830293685B1C93604268521C42604A68EF
:102B9000002ACFD061792079BDE8F0411047BDE827
:102BA000F04103487F3000F00FB80000C80000205B
:102BB0003D0405003807002002490F220A70886191
:102BC00070470000C8000020FFF7F6BF002100F0AA
:102BD00009B8012100F010B808B56A46FDF74DFBB1
:102BE000009808BD08B56A46FDF72DFB08BD08B57D
:102BF0006A46FDF70FFB08BD08B56A46FDF716FBF0
:102C0000009808BD08B56A46FDF744FB009808BD6A
:102C100070B5044600252846FDF781FE21686268EC
:102C2000086890420ED9401E08600178A38AE268C5
:102C300001FB0325227A2168101AC0B20A79824268
:102C400000D208710020FDF76CFE284670BD70B5FB
:102C500005460C460020FDF762FEE868A98A201AA6
:102C6000B0FBF1F12A681068431C13600170BDE8E5
:102C700070400020FDF755BE10B530B1017A4268B2
:102C80000368891AC9B21A6006E00E2010BD0368F5
:102C90001A68541C1C601170491EC9B2F7D2006832
:102CA00000210171084610BD70B5074C251F206832
:102CB00029684968884202D30448FFF785FF2868DD
:102CC00021688068405C70BD040100204400010060
:102CD00001480068704700000401002010B5044658
:102CE000054800684068A04202D80448FFF76CFF1E
:102CF0000148001D046010BD000100204C000100CF
:102D000001484068704700000401002010B50446E7
:102D1000054800680068A04202D80448FFF754FF45
:102D20000148001D446010BD000100205800010052
:102D300010B5040002D10548FFF746FF0448002102
:102D40000460001D0160416010BD0000270001000B
:102D5000000100200948021F4168491C41601268B7
:102D60001368994208D3002343600168491C01603D
:102D70005268914200D303607047000004010020B4
:102D8000002839D0401E00BF00BF00BF00BF00BFF9
:102D900000BF00BF00BF00BF00BF00BF00BF00BF3B
:102DA00000BF00BF00BF00BF00BF00BF00BF00BF2B
:102DB00000BF00BF00BF00BF00BF00BF00BF00BF1B
:102DC00000BF00BF00BF00BF00BF00BF00BF00BF0B
:102DD00000BF00BF00BF00BF00BF00BF00BF00BFFB
:102DE00000BF00BF00BF00BF00BF00BF00BF00BFEB
:102DF00000BF00BF00BFC5D170470000F0B5054659
:102E00000478154889B0164640F82420124A08690B
:102E10000832A2F10C0742F82400487F38552022DE
:102E20006846FDF77FFA04942878385C48B10EB103
:102E30000A4A00E000226946281D03F0BDFB09B0E4
:102E4000F0BD0EB1064A00E00022694605F10C0013
:102E500003F084FAF3E700000C000020616D00002D
:102E6000AD6B000070B5124D06464FF08074686877
:102E7000814202D01022FDF755FA0E490020C1F818
:102E8000000101220A6001E0641E0ED0D1F8002189
:102E9000002AF9D0C1F80001A9688E4203D010229F
:102EA0003046FDF73FFA012070BD002070BD0000E4
:102EB0001C00002000E000400549064801F1100216
:102EC000C0E900121032826003480160012070479F
:102ED000580100201C00002004E500400146024883
:102EE00010220068FDF71EBA1C0000202DE9F041F9
:102EF0000446102802D30B48FFF766FE094E0A4D20
:102F0000761D204600F07EF8070008D0AF4202D1BF
:102F10003046FFF759FE384600F03AF8F1E7BDE8D1
:102F2000F0810000D0000300ADDEADDE0148006896
:102F3000704700003401002010B50020114A0146FE
:102F400000EB40039C186170A170D154401CC0B2CA
:102F50001028F5D3DE22CC210B48FDF7F5F90A4AFB
:102F60000020A2F1180100BF00EB001302EB4303A5
:102F700041F82030401CC0B20628F5D30349062092
:102F8000086010BD2C090020340A00203401002004
:102F900070B5104C06462068062802D30E48FFF78D
:102FA00013FE3046FDF7DCFB18B90B48401CFFF759
:102FB0000BFE0A4D20680A4955F82000884203D0CC
:102FC0000548801CFFF700FE216845F82160491C78
:102FD000216070BD34010020800003001C0A002025
:102FE000ADDEADDE10B50446102802D30348FFF76E
:102FF000EBFD034904EB4400085C10BDC200030074
:103000002C09002070B500260446102802D30C4875
:10301000FFF7DAFD0B4D04EB4404285D70B105F1B8
:10302000300000EB8401601910F8022F51F8226083
:103030000321FFF7A5FA285D401E2855304670BDD4
:10304000A20003002C09002070B50C46064610298A
:1030500002D31248FFF7B8FD3046FDF781FB18B9DF
:103060000E48401CFFF7B0FD0D4D04EB4404285DF5
:10307000032810D205F1300000EB8401601910F82C
:10308000012F41F822600321FFF77AFA285D401CE6
:103090002855012070BD002070BD00008C00030089
:1030A0002C09002010B50446102802D30948FFF768
:1030B0008BFD094904EB44000A5C42B101F1300286
:1030C00002EB80020844807852F8200010BD0020F6
:1030D00010BD0000B30003002C0900200B4810B500
:1030E0000168002479B10A4A0A4B02EB8102491EA9
:1030F00052F8044D136001602046FDF731FB10B912
:103100000548FFF761FD204610BD00003401002096
:103110001C0A0020ADDEADDE7800030000487047D9
:1031200040A100402DE9F74F904607004FF0000501
:1031300002D13448FFF748FD334C4FF4803BC4F8CC
:1031400008B3324EB07818B12E48801DFFF73CFD11
:10315000706818B12B480930FFF736FDDFF8B0A0D2
:1031600077605FEA08004FF000094FF00108AAF10C
:10317000040724D001282FD0022829D021481D304F
:10318000FFF722FD86F80280C4F840910199294496
:1031900089B239603F68C4F84480DAF80060D4F836
:1031A000400118B117482B30FFF70EFDAF4215D381
:1031B000AE4201D3BE4221D3124833301CE0C4F8E2
:1031C0004480DAF80050C4F84080C4F84091D9E750
:1031D0000F48001D0568D5E73D68D3E7BE4201D220
:1031E000012000E00020B54201D8012100E00021CB
:1031F000884203D103483E30FFF7E6FCC4F804B32D
:10320000BDE8FE8F8600040000A000400C010020F5
:1032100044A500400048704748A0004070B5144CD9
:1032200001266660E6606664124800250560114864
:103230003C30006810B11048FFF7C6FC4FF0FF307B
:10324000C4F80803C4F840510A4904200831086052
:103250000A4845600670457085700A20FDF7D4F86D
:103260004FF0E0214FF48060C1F8000170BD000014
:1032700000A0004008A50040470004000C01002009
:1032800001480078704700000C010020034901202C
:1032900008600349002008707047000000A000404B
:1032A0000C01002070B5074801250561C560064C7A
:1032B00000260A2066606670FDF7A6F8A6702570E5
:1032C00070BD000000A000400C01002001484078C3
:1032D000704700000C0100200FB408B503990029C5
:1032E00004D004AA00926A4600F00FF801B05DF81D
:1032F00014FB10B582680446002A05D0D4E9040303
:10330000216898470020A06010BD2DE9FC47914638
:103310000C00804676D014F8011B39B125290ED057
:103320004046FDF729FC20780028F4D198F80C00DD
:10333000002867D04046BDE8FC47FFF7DABF002011
:10334000012221782B291BD02D2902D0302908D128
:1033500002E040F0010001E040F00200641C002A9D
:10336000EFD100252A290ED02178A1F130020A2AB6
:1033700011D205EB850201EB4205641C303DF1E7FB
:1033800040F00400EAE7D9F800100B1DC9F800303E
:103390000968641C0D44217800232E290BD114F8F0
:1033A000011FA1F130020A2A05D203EB830201EBCF
:1033B0004203303BF3E76C290DD068290BD0692913
:1033C00021D00BDC252918D0582931D063290ED003
:1033D000642915D117E014F8011FECE7702969D0B2
:1033E000732932D075291BD0782909D120E0D9F86A
:1033F0000000011DC9F8001001784046FDF7BCFB34
:10340000641C90E76CE0D9F800100A1DC9F8002090
:103410000968CDE900500A224046FFF7BBF8EFE704
:10342000D9F800100A1DC9F8002009680A2206E030
:10343000D9F800100A1DC9F8002009681022CDE94A
:103440000050404603F01EFDDAE7D9F800100027CF
:103450000A1DC9F800200E68C00705D112E04046D9
:10346000761C7F1CFDF788FB31780029F7D104E03A
:10347000202140466D1EFDF77FFBBD42C0D9002DC7
:10348000F6D1BDE74EB13046FCF770FF074604E0C9
:10349000202140466D1EFDF76FFBBD4206D9002D71
:1034A000F6D103E04046761CFDF766FB3178002933
:1034B000F8D1A5E7D9F80000011DC9F8001005688A
:1034C00030214046FDF758FB78214046FDF754FB7C
:1034D00008200021CDE90001034610222946B0E76B
:1034E000BDE8FC872DE9FF411C46DDE90A78154659
:1034F0000E46684600F07AF846EA450141EA840142
:1035000041EA072242EA0841009A00EB8200C0F833
:103510000017BDE8FF812DE9FF411C46DDE90A786F
:1035200015460E46684600F06FF846EA450141EA46
:10353000840141EA072242EA0841009A00EB820036
:10354000C0F80017BDE8FF812DE9FF411C46DDE909
:103550000A7815460E46684600F064F846EA4501CA
:1035600041EA840141EA072242EA0841009A00EB5D
:103570008200C0F80017BDE8FF811CB50021009152
:103580000B4601220191FFF7C6FF1CBD1CB50021AF
:1035900000910B4601220191FFF7D6FF1CBD1CB51F
:1035A00000220B46009211460192FFF7B4FF1CBDAA
:1035B0001CB500220B46009211460192FFF7C4FF92
:1035C0001CBD1CB5002100910B4601220191114642
:1035D000FFF7A1FF1CBD1CB5002100910B46012285
:1035E00001911146FFF7B0FF1CBD000001682029C2
:1035F00002D24FF0A040704701F01F010160014866
:1036000070470000000300500168202902D24FF0EB
:10361000A040704701F01F010160014870470000A1
:10362000000300500168202902D24FF0A0407047EB
:1036300001F01F01016001487047000000030050C5
:1036400001B56846FFF7E0FF009A01219140C0F8FC
:10365000081508BD01B56846FFF7E4FF009A01218F
:103660009140C0F8081508BD38B50124009068469F
:1036700031B1FFF7BBFF00998C40C0F8084538BD59
:10368000FFF7B4FF00998C40C0F80C4538BD00002E
:103690002DE9F041204D164688460746082801D3FB
:1036A000042035E0B8F1000F03D0202E03D9062006
:1036B0002EE003202CE0384601F086FA032801D3DF
:1036C000092025E0384601F013F8032801D30A2029
:1036D0001EE000F033FD022801D2082018E000F0BF
:1036E000BDFE044606704078324640F0010060702E
:1036F0004146A01CFCF716FEF8B2214601F066FA1E
:1037000010B10120BDE8F0810448FFF75DFA0F20F9
:1037100028700020F6E70000C8000020FC0005002B
:103720000149002048607047380700200348C16005
:10373000026101214170002181707047AE000020BC
:103740000348C1600261012141708170704700002F
:10375000AE00002010B500F0B5FD18B1BDE8104076
:1037600000F004B8BDE8104000F0AABC70470000AB
:1037700010B50B4C606928B100F05AFB0004000C36
:1037800002D005E0022008E0002000F071FE18B130
:1037900000F0AAFC012010BD11202070002010BDF7
:1037A000C80000202DE9F04116460F46044600F0FF
:1037B0009FFF154D48B157B1204600F0A5FF007896
:1037C0003168814205D206201AE00B2018E0032060
:1037D00016E0204600F08EFF04000DD0A01C0BD098
:1037E0002278A11C38463260FCF79CFD204600F090
:1037F0002BFE0120BDE8F0810448FFF7E5F90F201A
:1038000028700020F6E70000C8000020260105000F
:1038100010B5082804D3054904200870002010BD05
:10382000C0B200F05BFF012010BD0000C800002006
:10383000084910B54A69527D0AB10C2002E00828F7
:1038400003D304200870002010BDC0B201F0A4F919
:10385000012010BDC8000020014800697047000029
:10386000C80000200148007870470000C800002010
:1038700000F032BD082804D3034904200870401F1B
:10388000704700F035BF0000C800002001F0AAB862
:1038900001484068704700003807002001F0BAB8BE
:1038A00010B500F04BFCC0F1060010BD082804D391
:1038B000034904200870401F704701F085B90000DB
:1038C000C800002010B5012401F09AF9F02815D0A5
:1038D00005DCB0B1042809D0EC2812D110E0F4289E
:1038E0000AD0F82806D0FC280BD101E0002408E01B
:1038F000022406E0032404E0042402E0052400E09E
:103900000624204610BD70472DE9F0411D4D0646A6
:1039100000241D482C70AC610460446084601B4826
:1039200000F02EFC686140B3042000F09FFA05F11E
:103930001C00296900F086F80746304600F0D6F8EA
:1039400000EA0706002000F0B7F80640012000F06A
:1039500003F90640022000F097F80640002000F02E
:103960001DF90640012000F0A7FE0020EC6000F0E9
:1039700065FD16B10120BDE8F0810120287000200E
:10398000F9E70000C800002038070020352A0000B1
:1039900001484069407D7047C80000207047000022
:1039A00010B50446082803D30B490420087010E022
:1039B000FFF77CFF03280CDA2046FFF75BFF0328A4
:1039C00007DAFFF76DFFC0F10600022801D30120DE
:1039D00010BD002010BD0000C8000020084A10B52E
:1039E00053695B7D0BB1022002E0082803D3042059
:1039F0001070002010BD00F04BFD012010BD000034
:103A0000C8000020064910B54A69527D1AB102204B
:103A10000870002010BD00F011FA012010BD000058
:103A2000C8000020064910B54A69527D1AB102202B
:103A30000870002010BD00F00DFA012010BD00003C
:103A4000C800002010B50F4C6269527D0AB10220F7
:103A500014E010290FD871B178B10A4621610146EE
:103A600008481C30FCF75EFC064821691C3000F059
:103A700011FA012010BD072000E003202070002073
:103A800010BD0000C80000200A4910B54B6902466D
:103A900001205B7D0BB1022004E0012A05D0022A3F
:103AA00004D00E200870002010BD002000F070FA35
:103AB000012010BDC80000200A4910B54B6902461C
:103AC00000205B7D0BB1022003E032B1012A03D05C
:103AD0000E200870002010BD012000F0D5F9012053
:103AE00010BD0000C800002000F0FCBB10B540B1C4
:103AF000012808D002280BD00649052008700020B4
:103B000010BD012000E0022000F0F2FB012010BDFA
:103B10000020F9E7C8000020064910B54A69527D27
:103B20001AB102200870002010BD00F061FF0120D2
:103B300010BD0000C8000020064910B54A69527D3A
:103B40001AB102200870002010BD00F069FF0120AA
:103B500010BD0000C8000020014610B50020072954
:103B600014D2DFE801F0040F06080A0C0E0004204E
:103B700008E0FC2006E0F82004E0F42002E0F02059
:103B800000E0EC2001F042F8012010BD02490E20B7
:103B90000870002010BD0000C80000200A4910B5C0
:103BA0004B69024600205B7D0BB1022003E032B17D
:103BB000012A03D00E200870002010BD012001F062
:103BC0002FF8012010BD0000C800002010B5FFF73D
:103BD000DFFE002806D0FFF7BDFD30BFFFF7D8FE9F
:103BE0000028FBD110BD000038B50446012181F347
:103BF0001088202505E06A46064920460095FFF713
:103C0000D1FD2046FFF736FE0028F4DC002080F3CB
:103C1000108838BDFC06002010B501F0F3F9034907
:103C2000002008610249087010BD000090070020C4
:103C3000F40000202DE9FE434D4800684D4C01285A
:103C400002D04D48006828B960680078202801D863
:103C5000012100E00021494E03204FF000083070A0
:103C60004348C4F8008008300568424F183F89B3C4
:103C7000006841490839086002A8CDE900043C48C1
:103C80000C30026801232946184602F04FF910B3A0
:103C9000012805D0022821D0032855D0384851E00A
:103CA000029818B136481C38FEF78EFF284602F0FD
:103CB000A0FA18B932481B38FEF786FF01F0D6F992
:103CC000B97D0023CDE900017068EAB290F91610C1
:103CD00018461CE01EE02A48113833E0029818B953
:103CE00027480D38FEF770FF284602F082FA18B90F
:103CF00023480C38FEF768FF01F0B8F9B97DEAB245
:103D0000CDE900017068012390F91610029800F0C7
:103D10007DFB19E000F072FE30B101F0A7F9014619
:103D2000BA7DE8B200F044FB0023CDF800801A46CB
:103D300019461846CDF8048002F0F8F8042803D09C
:103D40000F480F30FEF740FF206838B10120607542
:103D50000C48206104203070BDE8FE8301F052F968
:103D600084F81580C4F8108000F00EF8F4E7000025
:103D7000001400409007002034150040F40000209B
:103D800044060900213E000070B5FFF745FF1F4DB6
:103D9000012028701E4801681E4A21F0FF011269A7
:103DA0001143016002F02EFA1A4C4C3410B302F0A9
:103DB00029FA032802D01848FEF706FF022001F076
:103DC0005FFB002001F0B4FB02F01CFA032803D0D3
:103DD00011480830FEF7F8FE2878012803D00E4875
:103DE0000E30FEF7F1FE02202870002020610B4803
:103DF000E06070BD02F012F80228DFD302F028F96B
:103E000060600028DAD10448401FD5E7F4000020A4
:103E10003015004044070020F4050900353C00003F
:103E2000024905200870FFF7AFBF0000F400002032
:103E30000148006A7047000044070020034910B59C
:103E4000086200F0ADFD0249086010BD4407002083
:103E50001C150040034910B5486200F0A1FD02495D
:103E6000086010BD44070020201500400449487731
:103E700004490A6822F4E02242EA004008607047E0
:103E800044070020181500400149087670470000DB
:103E90004407002070B50C00054602D10748FEF724
:103EA00093FE1DB90548401CFEF78EFE0448C0E98C
:103EB0000145BDE870400020FEF710BFB3030900C4
:103EC000A807002010B500F099FD044901F1640233
:103ED00008B1C86800E08868106010BD4407002081
:103EE0001CB510490320086002F08CF9012812D09B
:103EF000022810D0032813D1002000900346024668
:103F00000146019002F012F8042809D0BDE81C40D7
:103F10000548FEF759BE0021084602F0B7F8F3E75E
:103F20001CBD000008F5014048020900144981F851
:103F3000310014490A6822F0FF020A6048B1114AB0
:103F40000B1D0832012807D002280ED00E48FEF7BC
:103F50003BBE086808607047086840F001000860D0
:103F6000FF20106040F2071007E0086840F00200F0
:103F700008604FF6FF70106004481860704700003A
:103F800044070020341500402E04090021100100D0
:103F9000044981F83200044908B1012800D10860C1
:103FA0007047000044070020101500402DE9FF4134
:103FB0003E480068012802D03D48006830B93D48BD
:103FC00040680078202801D8012700E0002700F091
:103FD000F5FB384C0126183C00B9266102F012F9B5
:103FE000012802D03448FEF7EFFD344D6868007DAB
:103FF00018B13148401CFEF7E7FD01F003F8EFB3BC
:104000000121084602F042F820B1012828D00228F8
:1040100026D10FE001F02AF8064601F04FFFC7B2A3
:1040200001F046FF8446A07D0021CDE90260CDE984
:1040300000710DE001F01AF8804601F03FFFC7B2B1
:1040400001F036FFA17DCDE90076CDE902818446FD
:1040500068686289218990F91630604600F0B8F9E5
:10406000FEF736FEE06013484C3840696060FFF7A9
:1040700029FF04B00020BDE8F04100E001E0FEF7B8
:1040800045BE6E7000F0BAFC00280CD000F0EEFFC8
:10409000054601F013FFA27D04B02946BDE8F041BA
:1040A000C0B200F085B9BDE8FF81000000140040F7
:1040B000341500409007002037070900F400002065
:1040C00010B5012080F310880648417D29B1817820
:1040D00019B90121817000F03FFB002080F31088A6
:1040E00010BD00007807002070B5124C607D0028DC
:1040F0001ED100F0C3FA04F13005A86810B90E48CB
:10410000FEF762FD686818B90B48401CFEF75CFDBD
:1041100002F0A8F818B10848801DFEF755FD0020F0
:1041200002F0C0F801206075BDE8704000F014BBDB
:1041300070BD000078070020CE02090001F0CABE61
:1041400030B50D4D85B0687D002813D000F042FBDE
:1041500000F058FF0024AC706C7505208DF800004D
:10416000684601F007FE0548047005B0BDE8304020
:10417000FFF7B6BE05B030BD78070020F400002080
:104180002DE9F0410546012080F31088484E4FF09C
:1041900003080024707086F80080B4707460348165
:1041A0007481F46007463461347506F11800747543
:1041B000046044608460C4600461047518308460E5
:1041C0004460FFF72BF8284601F00EFE01F084FE54
:1041D000002002F059F806F13000FEF7A9FD002199
:1041E0000A20FCF73DF900210120FCF739F90121F3
:1041F0001420FCF735F9012000F07AF8A6F1340517
:10420000FF202861042068772A4929622A496962C7
:1042100085F82870022185F8291085F82A8085F80C
:104220002B00052085F82C00062085F82D0007209E
:1042300085F82E00082085F82F0085F8304085F895
:10424000311085F83270692045F8140B1E20286063
:104250004FF4167045F8100C022000F091FC0F206E
:1042600000F094FCEC802F716F712C72204601F0ED
:104270002BFE7078012802D01048FEF7A5FC37709D
:10428000B470746034817481F46034610C483475A6
:1042900074758460447000F0F1F90A20FCF7A9F805
:1042A0001420FCF7A6F884F310880148BDE8F081DB
:1042B0007807002004070A0D05080B0E9F0209006D
:1042C000F40000200348407D08B100207047012021
:1042D00070470000780700200148408B70470000BD
:1042E000440700200149488370470000440700202C
:1042F00010B5012181F3108807490A78824204D061
:104300004870487D28B100F027FA002080F310881B
:1043100010BD00F003F8F8E77807002030B5224D13
:1043200085B02878697888423BD008B900F0A6F9B2
:10433000687808B9FFF7D4FD1C480024046000F039
:1043400061FE194818300460446004618460C460F0
:104350002878012802D0022808D015E001F052FF89
:1043600090B10021084601F091FE0DE0FFF754FCEA
:1043700001F048FF032807D1002300941A4619468C
:104380001846019401F0D2FDFFF79CFD6878287073
:1043900004208DF80000684601F0ECFC012005B017
:1043A00030BD0020FBE700007807002014F5014035
:1043B00000B585B006238DF806208DF805108DF820
:1043C00004008DF80030684601F0D4FC05B000BD53
:1043D000F0B585B00DF1280C9CE8F0008DF80C309C
:1043E0008DF80D404FF0000C0190ADF808108DF8DD
:1043F0000E508DF800C0ADF80A208DF80F608DF8D2
:104400001070684601F0B6FC05B0F0BD70B586B01E
:104410000226DDE90A458DF808108DF80920019083
:104420008DF80A308DF800608DF80C508DF80B4037
:10443000684601F09FFC06B070BD0000014988602D
:1044400070470000F400002010B5012181F31088AE
:1044500001F068FD002080F3108810BD10B5012028
:1044600080F3108801F060FD002181F3108810BDF9
:1044700010B50446082802D30348FEF7A5FB0348FD
:10448000204490F8280010BDAD0309004407002027
:1044900070B5082819D20F4A024482F82810820702
:1044A000D40EFF22A240D243042801D20A4D01E0DB
:1044B000094D2D1D286810402860084600F05EFA5E
:1044C0002968A0400843286070BDBDE870400348DB
:1044D000FEF77ABB4407002024150040A70309001B
:1044E00010B51B4C00206070FEF7DEFB1949086018
:1044F000FEF7EEFB1849887501F084FE012807D00D
:1045000001F080FE022802D01448FEF75DFB002077
:1045100000F0B6FFFEF702FE114908606068091D51
:1045200040680860A068002811D0007820B1FEF72C
:10453000F5FDA16800F002FCA0680179002906D011
:1045400000F0D0FBA068BDE8104000F0D9BB10BD62
:10455000F4000020081500407807002097060900A5
:1045600010F5014010B501F0F7FD002820D01148EA
:1045700000210181418101F0A1FC0F49086001F097
:104580009DFC012181400C48001D026822F0FF02C1
:104590001143016001F08CFC064C1834206001F0DE
:1045A00081FC60600548E060BDE81040FFF798BFFF
:1045B00010BD0000780700202C150040AD3F000022
:1045C000154800210160012101601448016821F4AF
:1045D00080710160016821F00F01891D016001688F
:1045E00021F4702141F440310160001D016821F087
:1045F00000710160016841F080710160016821F083
:10460000FF0141F020010160016821F47F41016058
:104610000120FBF7EEBE0000FC1F00401415004017
:1046200070B5134C1348A16800F096FE6060114C01
:104630004C3C607FFFF71AFC206AFFF7FFFB606AC3
:10464000FFF708FC0025601990F828102846FFF7AE
:104650001FFF6D1C082DF6D3074914F8300F0860B2
:104660006078FFF763FCA078BDE87040FFF790BC6E
:10467000F4000020900700200C1500400C4910B5F4
:10468000002008600A4803240C380460FFF798FFF4
:10469000FEF7C0FD064908310860091F054808609B
:1046A000034810380460BDE81040FFF7B9BF0000B0
:1046B00014F501400411004010B504460448406858
:1046C00010B90448FEF780FA0348047510BD0000D5
:1046D000F40000206E0409009007002010B50121AD
:1046E00081F3108801F082FD002080F3108810BD56
:1046F00001F07FBD10B5012181F3108801F07CFD30
:10470000002181F3108810BD01F079BD0349012219
:10471000086101460248FEF705BD00007807002049
:104720007162000070B50C4601F0BCFD074D2869B0
:10473000A04202D30648FEF747FA28690122211A4F
:104740000448FEF7EFFC0020286170BD78070020C8
:10475000D60609007162000010B5FEF791FD012830
:1047600022D101F099FD10B11048FEF72DFA002278
:1047700064210F48FEF7D6FC0E48007F80B90E4832
:104780000121016000220007C0F80021016000BF84
:1047900000BF00BFAFF30080D0F800110029FBD0AC
:1047A000BDE81040FEF772BD10BD0000B406090060
:1047B000716200004407002014050040044810B551
:1047C000006918B9FEF782FD002800D0012010BD55
:1047D0007807002010B5FEF753FD01280ED0FEF734
:1047E00061FD0748007F10B9012081074860002063
:1047F00001F058FD024900203431486010BD00002E
:10480000440700200B4810B54068407D30B10120BE
:1048100000F08EFE08490889401C088107490020E5
:1048200008600548343803C8BDE81040091A002064
:10483000FFF778BFF40000207807002014F501404E
:1048400070B586B0FFF7BAFF494D4A4E05F1340402
:1048500058B100F0BDF8A078002869D0FEF77AFAC8
:1048600006B0BDE87040FFF76BBC2078012802D08D
:10487000022804D008E000F017FF28B170E030787B
:1048800004286DD003286BD0FEF764FA00F0A0F87E
:10489000A07868B1FFF754FC01F0C0FA022840D3B9
:1048A00003208DF80000684601F064FA06B070BD80
:1048B000FFF734FD20B100206968FFF733FFEBE715
:1048C0002078F0B1012816D0022817D02A48FEF728
:1048D0007BF9687E0128DFD100F090F80028DBD159
:1048E0002078D8B1012811D00228D5D022481A301A
:1048F000FEF76AF9D0E700F099F8EAE700F01AF954
:10490000E7E700206968FFF70DFFE2E701F07AFCB6
:104910000028C1D101F0F4FB0028BDD1FFF75AFFF8
:10492000BAE706B01448BDE870403630FEF74CB91F
:104930002078022808D0FEF70DFA696806B000203A
:10494000BDE87040FFF7EEBE3078042808D0032899
:1049500006D0FEF7FFF906B0BDE8704000F0EAB8F7
:10496000686806B04008BDE87040FFF7CFBE0000A1
:1049700044070020F4000020D0040900024610B5CE
:104980000020014622FA01F303F00103C1F10704FC
:10499000A3400343491CC9B2D8B20829F2D310BDC1
:1049A0002DE9F0410024064625461827E80026FA9E
:1049B00000F0C0B2FFF7E2FF694207EBC101884097
:1049C00020436D1CEDB20446042DEFD3BDE8F08109
:1049D0000348416809B1491E4160FFF773BA0000FE
:1049E0007807002001484069704700004407002014
:1049F00001494861704700004407002004480178DD
:104A0000022902D04068002800D001207047000031
:104A100078070020014840687047000044070020E4
:104A20000149486070470000440700202DE9F0412B
:104A300086B000F0E7FA01F0E5FB3A4D05F13404E9
:104A400020B3688BB0B3218981423BD30121002080
:104A500001F01CFB01F02CFA26898046648901F0E4
:104A60002DFA074600F002FB014601208DF80000F8
:104A7000ADF808608DF80C70CDF80480ADF80A40F0
:104A80008DF80D10684601F075F944E001F0C6F9A3
:104A9000022840D3FFF7B2FF68B1FEF731F9D0BB6F
:104AA000287E20B9FEF714F9E168884233D1FFF778
:104AB00059FD30E006E0E068FEF710F90020FEF74F
:104AC00025F9F4E7FEF702FC10B11748FEF77CF871
:104AD000FEF7EAF815490968884202D06089401C4F
:104AE000608113484078A0B9FFF788FF88B101F0D2
:104AF000E5F9064600F0BAFAA17D8DF806108DF8AA
:104B0000050007228DF800208DF80460684601F04A
:104B100031F9FFF7E5FC296806B00120BDE8F04156
:104B2000FFF700BE440700207C050900081500407F
:104B3000F400002070B50024FEF7B6F80D4D29688A
:104B4000884207D0FEF7B0F82860FEF7C1F80A499E
:104B5000012488750948641E0078044201D1FFF7DA
:104B600013F9054834384168BDE870400020FFF76C
:104B7000D9BD00000815004078070020F40000208F
:104B80000149C860FFF79EB94407002001498860C9
:104B9000FFF798B94407002010B50446012181F3BE
:104BA00010880748017821B1407D10B10548FEF713
:104BB0000BF8204601F02CFB002080F3108810BD7C
:104BC000780700206803090001F02BBB10B5012213
:104BD00082F3108801F032FB58B10848817819B986
:104BE000407D08B1FFF7B8FD002080F31088012058
:104BF00010BD002080F3108810BD00007807002051
:104C0000014890F83000704744070020024981F8BD
:104C10003000024908607047440700200C1500402E
:104C200001490877704700004407002070B511491A
:104C3000114A0025487802EB0010027B22B10F4A8E
:104C4000D2F80C2102B10125807A0870012000F011
:104C5000DFFB0B4C1DB1A068806800B18047606825
:104C6000002806D00179002903D0BDE8704000F08B
:104C70001BB870BDB4070020A86F000000100040F2
:104C80001401002007480069012805D0022805D03A
:104C9000032805D100F09AB800F04CB900F0E4B850
:104CA00070470000B4070020827B002193000B4A6C
:104CB0001344C3F81019C37B02EB8302C2F8101926
:104CC000427B0121837BC07B01FA02F201FA03F3EC
:104CD000814003481A430A430260704700F00140D4
:104CE00008F501404279054BC079012103EB8000B2
:104CF0000AB1016670470163704700000060004020
:104D000082680021C2F84011C17B094ACB000949E1
:104D10000B44C3F81025C37B826801EBC301C1F8C3
:104D20001425C17B012088400349086070470000BA
:104D30001011004000F0014004F501402DE9F04160
:104D40000746886800260C46C0F840618868097BE1
:104D50001A4D00F5A07005EBC101C1F8100562788D
:104D6000E178207B00F08EFC607B05EBC000C0F892
:104D70001075617BA06805EBC101C1F814051048EE
:104D8000C0F80C61C0F81061A17B0E4805EBC101B1
:104D9000C1F810056278E178A07B00F061FC217B0E
:104DA0000120627B00FA01F100FA02F21143A27BBA
:104DB0009040014304480160BDE8F08100F00140EB
:104DC000001000400C11004004F501402DE9F041B5
:104DD0001F4E0220002530700320707075603575FD
:104DE000B0691C4C401CB061C4F80C51C4F80051AF
:104DF000C4F81051C4F80451C4F82851C4F8005242
:104E0000681EC4F808030120FBF709FB124FB868BD
:104E1000007D50B1114800684042B075C4F81C5183
:104E20000120A0610E49042008600C484438006845
:104E3000F168884202D00B48FDF7C6FEB868C0682A
:104E4000002802D0BDE8F0410047BDE8F081000035
:104E5000B407002000100040140100204815004055
:104E600008F5014051040A0010B52D4CD4F80C018E
:104E7000012802D02B48FDF7A7FED4F81001012825
:104E800003D02848401CFDF79FFED4F800010128FC
:104E900003D02448801CFDF797FED4F8040118B114
:104EA0002048C01CFDF790FE0020C4F80C01C4F897
:104EB0001001C4F80001C4F80401C4F8080102217B
:104EC000C4F800120121C4F808130822C4F804230E
:104ED000154A0323154C137010755060606890B12B
:104EE000027912B1FFF7E0FE0DE002785AB1027BC1
:104EF000437B807B01FA02F201FA03F381400C4804
:104F00001A430A430260A068006900B18047A068A4
:104F10008068002802D0BDE81040004710BD0000A6
:104F200000100040F3030A00B40700201401002021
:104F300008F501402DE9F0412A4DD5F8000101287E
:104F400002D02948FDF740FED5F80401012803D01E
:104F50002548401CFDF738FE2448016824480170AC
:104F60000021C5F80011C5F80411C5F80811491E43
:104F7000C5F808130126C5F8046381681D4F097D33
:104F800009B104213960446814B3207900B3617B0E
:104F9000DFF86480A06808EBC10100F5A070C1F8DB
:104FA00010056279E179607B00F06CFB607B06FAAA
:104FB00000F03860207B114908EBC000C0F81015E4
:104FC0006279E179207B00F04BFB207B86403E60DC
:104FD0000B480649091FC06808600B20C5F800028D
:104FE000BDE8F08100100040BD030A000815004034
:104FF0001401002004F5014000F001400C110040B4
:10500000B407002070B50120FBF714FA0120FBF76C
:1050100006FA144C4FF0FF30C4F808030026C4F819
:105020000062C4F8106101202061A0610E4D287853
:10503000012813D0022813D0032811D05FF00100FB
:10504000FDF79EFEC4F810612E706E75002000F012
:10505000DFF9BDE870400120FBF7F7B90620EFE764
:105060000220EDE700100040B4070020014800785E
:10507000704700001401002001F03F014FF400339D
:1050800043EA0121830009481844C0F81015D0F8FC
:1050900010150AB941F48011C0F81015D0F8101598
:1050A00041F00301C0F81015704700000060004097
:1050B00008480069012806D0022806D0032806D037
:1050C0000548FDF781BD00F095B800F007B800F085
:1050D000F1B80000B407002033050A002DE9F047BD
:1050E000DFF8F0804FF00409012088F80090D8F82C
:1050F0001810491CC8F81810FBF791F936480068D9
:10510000364D2870364C0026C4F80C61C4F8006196
:10511000C4F81061C4F80461A868DFF8C8A00127CA
:10512000007D90B12F4808380068400702D42E480F
:10513000FDF74AFD284840300068404288F81600D4
:10514000C4F81C61A761CAF80090D4F8000118B136
:1051500025480930FDF738FDD4F80C0118B1224874
:105160000A30FDF731FD4FF0E020B046D0F80002E4
:1051700010F0020F03D01C480B30FDF725FD6E68C0
:10518000CEB13078B8B1C4F80C81717B184A174899
:1051900002EBC101C1F810057278F178707B00F064
:1051A0005FFA707B0F4907FA00F0091F0860F07B77
:1051B0008740CAF80070A868C06800B18047A86836
:1051C000417D002903D004490068091F0860BDE83B
:1051D000F0870000B40700200815004014010020EB
:1051E0000010004008F50140C0040A000C11004006
:1051F00000F001402DE9F041294C0026C4F80C6173
:10520000C4F80061C4F81061C4F80861C4F804610E
:10521000012004F58074FBF702F90820C4F80402A9
:105220000125C4F808520720C4F800011D4844684D
:10523000002C32D0207920B1207B1B4905FA00F0E8
:1052400008602078002828D0A068C0F84061A17BC1
:10525000164FA06807EBC10100F5A070C1F810055A
:105260006278E178A07B00F00DFAA068C0F8406198
:10527000E17B0F4807EBC101C1F81005E17BA06895
:1052800007EBC101C1F81405A17B05FA01F0E17B30
:105290008D4005492843091F0860BDE8F0810000E2
:1052A000001000401401002008F5014000F001400A
:1052B0000C11004070B5234CD4F80C01012802D029
:1052C0002148FDF781FCD4F81001012803D01E48C5
:1052D000401CFDF779FCD4F80001012803D01A48DE
:1052E000801CFDF771FC0020C4F80C01C4F810010B
:1052F000C4F80001C4F80401411EC4F80813C4F83E
:105300000002124C626872B1117861B1557B0123C1
:1053100003FA05F1957BD27B03FA05F593400C4A1D
:105320002943194311600B49032208704A704860F1
:105330000875A0680069002802D0BDE870400047E9
:1053400070BD000000100040F5040A0014010020A8
:1053500008F50140B407002070B506460C46012050
:10536000FBF768F8FFF74EFE244D25482649C5E9AE
:1053700001460024047003264670446004610475ED
:10538000447584751F4808601E48F030091F086086
:105390001E48016821F0010141F080710160012087
:1053A000FBF753F8686838B3017909B9017819B384
:1053B0008168C1F808650422C1F81025027CC2F199
:1053C0008102C1F8402540F20112C1F80022C1F863
:1053D00004450122CA60C1F84041017921B14279F6
:1053E0008179C079FFF748FE6868017821B1427879
:1053F0008178C078FFF740FE014870BD140100209D
:10540000B40700201410004024F501407417004038
:105410002DE9F041174C00250746C4F80052164EFE
:10542000307803281CD0681EC4F80803C4F80C5157
:10543000032070700120FAF7F2FF00BFC4F800519A
:10544000C4F81051C4F8045175603575002F0FD0A1
:105450000A488068006900280AD0BDE8F04100478A
:105460006FF00800C4F808030820C4F80403E5E757
:10547000BDE8F08100100040B407002014010020B6
:105480002DE9F0470746DFF8908022484FF0FF31C2
:1054900000EB0716C8F808130120FAF7C0FF1F4CED
:1054A0000025DFF87C9065756770D9F80800032F38
:1054B0000268A2604168C4E90315A56130686060B4
:1054C00019D2337AC8F80032C8F80C51C8F8105114
:1054D000F37A14481BB10160006828B108E002604B
:1054E000006828B9104801E00F48401DFDF76CFB2B
:1054F000717AC8F80413D9F80800007D28B1022F8A
:1055000003D10A49A5750420086001206075BDE833
:10551000F0870000A86F000000100040B4070020D2
:1055200014010020041500409C020A0004F501400B
:105530002DE9F05F404C82464048667800EB061744
:10554000607D012802D03E48FDF73EFB207D18B16A
:105550003B48401CFDF738FB012500212575DFF88D
:10556000E490A0466175032E47D2BAF1000F3CD1FA
:10557000D9F80440BCB32279AAB38A460846A16888
:10558000C1F84001217BDFF8C0B0A0680BEBC1017E
:1055900000F5A070C1F810056279E179207B00F078
:1055A00071F82A49C1F80CA1607B29490BEBC000B6
:1055B000C0F810156279E179607B00F051F8217B29
:1055C000627B05FA01F005FA02F1084321490860FF
:1055D000D9F80400204A81791268CA4012F0010FFC
:1055E00001D18068056038680560022E01D0012E67
:1055F00007D1B97A88F8001003E011482530FDF78B
:10560000E3FAD9F80800007D002813D0022E11D14A
:1056100010480068400703D409482A30FDF7D4FA3F
:105620000E480068002805D1BDE8F05F04482B3023
:10563000FDF7CABABDE8F09FB4070020A86F0000CC
:10564000B8020A001401002000F0014000100040E0
:105650000C11004004F501401005005004150040F5
:10566000064B03EBC0000AB1054A01E0044A303A98
:1056700002EB8101C0F814157047000000F00140F2
:1056800060600040064B03EBC0000AB1054A01E030
:10569000044A303202EB8101C0F814157047000053
:1056A00000F00140306000400348D0F804010128B8
:1056B00000D00020704700000010004030B5124BB1
:1056C00001460020D3F81044224609E0157A8542AD
:1056D00005D1401C0A28F7DB4FF0FF3030BD52687F
:1056E000002AF3D1421CF9D00872D3F810242AB151
:1056F00052684A60D3F81024516030BD0022C3F8CC
:1057000010144A6030BD0000D8020020F0B595B0FA
:105710001C4615460F4608461A9E00F009FB182144
:1057200009A8FAF718FE0E96CDE9095400230822BD
:1057300003A9384600F011FB05980690BDF810004B
:10574000ADF81C00BDF81200ADF81E0000208DF869
:1057500021000398082600F00300012802D0022847
:1057600018D032E003983346850AC0F3C2008DF8A2
:10577000200003980FA9C0F38314A200384600F05C
:10578000ECFA09A8009006AB22460FA9284600F0C3
:105790002BFA1AE00398840DC0F3C2008DF82000A4
:1057A000082C01D2254600E0082533462A460FA9D9
:1057B000384600F0D2FA2E44641B09AB06AA2946EB
:1057C0000FA800F063F9002CEAD1384600F0B6FAD1
:1057D00015B0F0BD7047012001F006BA084810B5B9
:1057E0000178084A515C19B1001D00F071FF02E018
:1057F0000C3000F07FFEBDE81040002001F0F4B94D
:10580000380000200800002008B5034A0092402319
:10581000024AFFF77BFF08BDA56A0000D8010020FF
:105820000A4A012902EBC00007D0022907D0032948
:1058300007D0042907D000207047022070470420B9
:10584000704700797047407970470000147100007C
:1058500010B5FFF7C0FF04210348FFF72FFF0249EF
:105860000120487210BD00004C0000202DE9F047D7
:105870008CB0FBF791F918B100200CB0BDE8F087AF
:10588000784C0020C4F81804BFF34F8F6068029072
:10589000A5684FF00008284004EB800008E021686C
:1058A0000298814201D86160E6E7284004EB80005D
:1058B0000C3002A9FCF702FF0028F0D103AB0299DB
:1058C00001EA050204EB8202491CD26843F8202059
:1058D000401C02910228F2D3039800F00300022832
:1058E00002D001284ED0A5E003985022810D8946B0
:1058F000B2EB905F00D850210E4666F39F500390A4
:105900000831594800F0CBF9070078D000F010FAC0
:105910004346082203A9384600F025FA029908F107
:10592000080A2940681A8000001D864223D94D4D7F
:105930000C3530B1C2B204EB8101301A90460C3103
:1059400004E02946F2B2002590462846C6B25346E6
:10595000384600F008FA0AEB08032DB13246294612
:105960004FEA070000F0FFF9029909F1030001EB8B
:10597000900002903AE004EB8101534632463846EB
:105980000C31EFE70398C0F38311062900D30621F9
:1059900061F389100390C0F38310801C81003248AA
:1059A00000F07DF9070045D000F0C2F94346082217
:1059B00003A9384600F0D7F908F1080800260FE0DF
:1059C0000298434600EA0501401C04EB8101029065
:1059D000042238460C3100F0C6F908F10408761CA0
:1059E0000398C0F38310B042EAD847B1D4F81054FA
:1059F000D4F8180468B1384600F0A0F92CE019E09A
:105A0000687A012804D12A682846394612689047E6
:105A10006D68002DF4D1384600F090F90020FAF7B7
:105A20007EFFD4F8180408B9029860600020FAF7E5
:105A300078FF11E0D4F8104404E02168204689681A
:105A400088476468002CF8D108480221008801EBDF
:105A5000004007A100F016F8FBF79EF880F0010067
:105A60000BE70000D80200203C7100004801002034
:105A70004261636B656E647320666C757368656400
:105A80000000000000231A4601F02CB82DE9F04771
:105A90000E4680461C46924608293ED894F80C9043
:105AA000002020731946104600F0C8FE0025B542BC
:105AB00006D218F805201AA12046FDF70DFC03E0D8
:105AC00019A12046FDF708FC6D1C082DEFD317A186
:105AD0002046FDF701FC0025B54210D218F80570EC
:105AE000FAF71CFC0068C05D10F03E0F01D03A468A
:105AF00000E02E220EA12046FDF7EEFB03E00DA1F3
:105B00002046FDF7E9FB6D1C082DE5D30122214657
:105B1000504600F075FE84F80C90BDE8F087000058
:105B20002025303278000000202020007C0000007A
:105B30002563000020000000104810B5FF2181609F
:105B4000002101604160C0F81814C0F8141480F8F6
:105B500020140B4800F0F0F800280DD109480A493C
:105B60000A4B401AC108002003E000BF23F82000C0
:105B7000401C8842FAD3002010BD0000D80200204B
:105B80003C7100003C7100001471000038010020DD
:105B900002480349401AC008704700003C710000E9
:105BA0001471000013B56846FCF7DAFE08B1002056
:105BB0001CBD0248009950F831001CBD1471000052
:105BC00070B508480125D0F8104480F8205405E04D
:105BD000657221682046496888476468002CF7D1BF
:105BE00070BD0000D80200202DE9FF4781460C9DC2
:105BF00000200C462F7B28739846164629461846E7
:105C000000F01CFE072E42D2DFE806F004090F1652
:105C10001F2A360049462846FDF75EFB37E0494615
:105C200028462268FDF758FB31E0D4E900234946B5
:105C30002846FDF751FB2AE0A0680090D4E9002334
:105C400049462846FDF748FB21E0D4E90201CDE9A9
:105C50000001D4E9002349462846FDF73DFB16E044
:105C600004F1080007C88DE80700D4E9002349467D
:105C70002846FDF731FB0AE004F108000FC88DE863
:105C80000F00D4E9002349462846FDF725FB0022F2
:105C90002946404600F0B4FD2F73BDE8FF872DE98B
:105CA000F041858A80462D1F4819C01CB0FBF5F0D5
:105CB000C6B24046FCF7ACFF041E19D0002020718C
:105CC00001206071E58000272546761EC4F800801B
:105CD0000BE04046FCF79CFF60B16179491C6171A3
:105CE000286005467F1CC0F80080B742F1D32046EB
:105CF000BDE8F081204600F002F80020F8E72DE929
:105D0000F041457901466B1E002201E00968521CF2
:105D10009A42FBD30F680146002605E038460C681E
:105D2000FCF795FF2146761CAE42F7D3BDE8F08123
:105D30000121001DFCF750BFFCF79EBF10B50446C3
:105D40000121001DFCF75EFF10F0FF0F04D120467B
:105D5000BDE81040FFF7D3BF10BD38B50124009453
:105D6000FCF7C2FD38BD38B500240094FCF7BCFD3B
:105D700038BD000070B51A4C0546206810B91948A6
:105D8000FCF722FFD4F8D4000A2803D31548401C9E
:105D9000FCF71AFFD4F8CC0000EB800004EB800184
:105DA00015F8040B08712DCD8860CA600B614D6138
:105DB000D4F8D400401CC4F8D400D4F8CC00401C63
:105DC000C4F8CC00D4F8CC1000200A2901D3C4F8C0
:105DD000CC004FF0E0214FF48010C1F8000270BDFC
:105DE000D00700204A000B0010B5040002D109487A
:105DF000FCF7EAFE084941F8CC4B002041F8740951
:105E00008867C8674FF0E0214FF48010C1F80001A7
:105E100010BD00003E000B00D007002010B5074C5D
:105E2000D4F8D4000A2802D90548FCF7CDFED4F8EE
:105E3000D400C0F10A00C0B210BD0000D00700209D
:105E400079000B0010B500F003029043D200FF244C
:105E5000944003689140A343CA18094901230B6089
:105E6000BFF36F8FBFF34F8F026006480268002AAE
:105E7000FCD000200860BFF36F8FBFF34F8F10BDC1
:105E800004E5014000E40140F0B515460E46074622
:105E9000002404E0315D3819FFF7D4FF641CAC42E4
:105EA000F8D3F0BD0148C06870470000A808002082
:105EB0000148806870470000A80800200148406839
:105EC00070470000A8080020014981F88100704750
:105ED000A8080020FDF72AB870B5FDF72DF80024BA
:105EE0000E4E2546204600F04BFC04F1080000F061
:105EF00047FC3555641C082CF4D309480121057072
:105F000045608560C5600561456180F8805080F816
:105F10005850C56780F8811070BD00002001002036
:105F2000A8080020FDF734B8FDF7D8B82DE9FF4FD9
:105F300081B0444FDDE90EA803260025F86F0C461A
:105F4000AB4610B94048FCF73FFE3878032803D031
:105F50003D48401CFCF738FEF86FB9464178C80749
:105F60002FD199F8810060B300270198E8B3039A14
:105F7000584662F31700C1F3410161F31F6009EB5A
:105F800084018A6BCAF800B0C8F800B00090904253
:105F900034D0204600F01CFC051E07EA05072DD072
:105FA00004F1080109EB81020099916104990D4205
:105FB00023D0264E305D00B3204600F032F910B1F8
:105FC00005E00127D1E720482830FCF7FDFD2046F9
:105FD00000F029F9CAF80000BAF1000F0AD018B988
:105FE00019482E30FCF7F0FD00E01BE006F804B085
:105FF000022603E014483230F4E7012677B1204648
:1060000000F02DF9C8F8000018B110480121015521
:1060100006E00C485830C8F8000001E0C8F800B0AD
:106020000DB107E004264C46D9F87C00FCF7B0FF20
:10603000C4F87CB089F800B000F068F805B03046CC
:10604000BDE8F08FA80800202D010C0020010020E1
:1060500010B50C4C207810B10B48FCF7B5FD00F0E2
:10606000ABFB00280DD0FF220270417841F0060101
:10607000417000214318491C9A702029FAD303214A
:10608000217010BDA808002007010C0070B51A4C43
:1060900005460E462078012804D0022802D0174871
:1060A000FCF792FDB5B12078012803D01348401DBC
:1060B000FCF78AFDE06818B91048801DFCF784FDE4
:1060C000E068007820B1606800F082FB022502E001
:1060D000002500E004254EB1606800F0A4F8A16836
:1060E000814203D005481D30FCF76EFD0020207072
:1060F00000F00CF8284670BDA8080020CC000C0069
:10610000014890F880007047A80800202DE9F04170
:10611000104C207800281AD194F88000002816D15D
:106120000825012600276069FCF75CFF18B184F898
:106130008060606920616069401C6061082800D14E
:10614000676194F88000002801D16D1EEBD1BDE895
:10615000F0810000A808002070B5224C207810B112
:106160002148FCF731FD94F880000025F8B1206942
:10617000606000F074F8A06018B91B48C01DFCF7FF
:1061800023FDA0684078C00705D194F8810010B1C4
:106190000220E56009E0606800F02BF8032806D2D1
:1061A00000F00AFBE06010B10120207002E02078CE
:1061B000002815D0A06818B90B482030FCF704FD62
:1061C0002069606004EB8000C17E491CC17684F8C0
:1061D0008050C27EA068417862F342014170012084
:1061E00070BD0000A808002098000C000830FCF7E3
:1061F0007DBE0830FCF7F6BE0830FCF703BF083060
:10620000FCF750BF0148007870470000A808002044
:1062100010B5044600F0BCFA2046BDE81040FCF77B
:1062200065BEFCF7DFBE70B50446FCF7EBFE05006B
:1062300002D0204600F0ACFA284670BD70B50E467C
:1062400004460025FCF772FE38B121463046FCF7C3
:10625000FBFE10B1FFF75AFF0125284670BDFCF781
:1062600021BF00000148007870470000280100208D
:1062700004480178817041780170001D50F82100B8
:10628000004700002801002002498870487008700B
:106290007047000028010020014840787047000046
:1062A0002801002010B50446022802D30248FCF75A
:1062B0008BFC0248447010BD33000D002801002003
:1062C0004058002800D00120704708B500224250F5
:1062D0004058009008BDD0F80403084000D00120C9
:1062E00070474058002800D00120704708B50022B0
:1062F00042504058009008BD0121B1EB507F01D1C0
:10630000012070470020704770B50D4600F0E2FA9A
:1063100004000FD00020FAF702FB207920B1002002
:10632000FAF7FFFA112070BD0120256020710020CE
:10633000FAF7F7FA002070BD10B500F0CBFA00288C
:1063400002D000210160017110BD00000149024826
:1063500000F072BC88010020002000402DE9F041CF
:106360000546007916460F4600EB40012D4A01EB29
:10637000C00102EB810494F82A1011B10820BDE895
:10638000F081294951F820102868FFF7BDFF08B1B6
:106390001120F4E739462846FAF7D8FA66603869DA
:1063A000206030004FF001062FD03F7F4FF48E71F8
:1063B0002868FFF78AFF4FF4A2712868FFF785FF6E
:1063C00028681A49C0F8041328684FEA4711000BDF
:1063D00040B2002806DA00F00F0000F1E02080F85B
:1063E000141D03E000F1E02080F800142868000B81
:1063F00040B200F01F0206FA02F14009800000F1ED
:10640000E020C0F88012C0F8001128680421C0F80C
:1064100000150020A061E06184F8290044F8140F01
:10642000A675ACE788010020406F000080000200E4
:106430002DE9F047054600790B4600EB400101EBE2
:10644000C000234901EB8004284600F043F810B156
:106450001120BDE8F0874FF00008C4F82080A36049
:10646000626184F828804FF48E764746314628686A
:10647000FFF72BFF28684FF00109C0F8089021466C
:10648000286800F075FB606800BBD5F800A00EE03E
:1064900094F8280008B10F2716E031465046FFF760
:1064A0000FFF0028F4D02146504600F061FB216A1E
:1064B00060698142F1D331462868FFF701FF002867
:1064C000F9D02868C0F80C90C4F814803846C0E7AA
:1064D00088010020007900EB400101EBC000044975
:1064E00001EB80004069002800D0012070470000C7
:1064F000880100202DE9F047044600794FF000099B
:1065000000EB400101EBC000254901EB800720684A
:10651000C0F80095786880B120682249C0F8081357
:1065200020680121000B40B200F01F029140400999
:10653000800000F1E020C0F880112068D0F80C2520
:10654000D0F81485D0F80865D0F810554FF0FF3119
:10655000C0F81415C0F80C152068C0F80815C0F86C
:106560001015501C02D01046FDF707F8B8F1FF3F98
:1065700002D04046FDF701F8681C02D02846FCF71F
:10658000FCFF701C02D03046FCF7F7FF2068FFF7D5
:10659000D3FE87F82A90C7F80490BDE8F087000082
:1065A00088010020840202000149024800F0F0BB8B
:1065B000B4010020002000402DE9F04105461646B8
:1065C00000790F46154A00EBC00102EB810494F8F4
:1065D000201011B10820BDE8F081114951F82010B8
:1065E0002868FFF791FE08B11120F4E739462846E4
:1065F000FAF7E7F96660386920601EB1397F2846EE
:10660000FCF71CF828680821C0F800150020A061DC
:10661000E0610121606184F82010DCE7B401002012
:10662000446F00002DE9F04704460E4600792049EA
:1066300000EBC00001EB800517463046FFF75CFE1B
:1066400030B1204600F036F820B11120BDE8F087C7
:106650001020FBE76F61AE604FF490760027314663
:106660002068FFF743FE4FF4AC7841462068FFF7FF
:106670003DFE2068AA686969C0F84425C0F848153D
:10668000206801218160686878B9B1464946206870
:10669000FFF727FE064641462068FFF722FE064325
:1066A000F4D000B10F27002068613846CEE7000023
:1066B000B40100200079054900EBC00001EB800027
:1066C0004069002800D0012070470000B40100207C
:1066D0002DE9F04704460079274900EBC00001EBA3
:1066E000800720684FF00009C0F80095786880B1F5
:1066F00020682249C0F8081320680121000B40B22D
:1067000000F01F0291404009800000F1E020C0F835
:1067100080112068D0F80C25D0F81485D0F80865D1
:10672000D0F810554FF0FF31C0F80C15C0F8141513
:106730002068C0F80815C0F81015501C02D010468B
:10674000FCF724FFB8F1FF3F02D04046FCF71EFFE4
:10675000681C02D02846FCF719FF701C02D0304696
:10676000FCF714FF2068FFF7E7FD87F82090C7F8D3
:106770000490BDE8F0870000B4010020100302007F
:10678000024A002102EB800081617047A8080020C6
:1067900010B50446064890F8801021B10069A04267
:1067A00001D1FFF7B3FC03490020085510BD0000DC
:1067B000A80800202001002010B5044CE06F00283C
:1067C00002D1FCF78BFCE06710BD0000A808002098
:1067D00070B5094D0446E86F10B90848FCF7F4F9A4
:1067E00004F10801E86FFCF72FFC002802D000201C
:1067F000E867012070BD0000A80800202E020C00F0
:1068000010B50C46017A052908D0407A38B10848FD
:1068100008A102682046FCF75FFD00E01AB106A15E
:106820002046FCF759FD2046BDE81040FCF761BD4D
:1068300084000020257300000D0A000038B5C388CD
:106840000D46044633B114A0009015A216A12846A7
:10685000FCF742FD217A05291CD0607A48B1A08856
:10686000FEF7DEFF164951F8202016A12846FCF756
:1068700033FDA0880021FFF795F903461049207ADF
:10688000143951F8202001B02846BDE830400EA14F
:10689000FCF722BD38BD00001B5B306D000000001E
:1068A0001B5B313B33316D0025734C6F6773206484
:1068B000726F70706564202825642925730D0A00A5
:1068C00084000020257300003C25733E2025733A88
:1068D000200000000349884201D10348704700208E
:1068E0007047000000200040280000207CB568466A
:1068F000FBF713FF294C20786178084302D1FAF79F
:10690000CBF96070607821784FF0010688434FF032
:1069100000050BD0FBF7A4FB012831D0022801D0E1
:10692000032801D1257065700028F3D02078A17864
:10693000884305D008216846FAF77CFA18B3A67098
:106940002078A178084228D008216846FAF772FA20
:10695000134A03210028108801EB004015D011A133
:10696000FFF790F80020FAF7B6F80028FAD1684649
:10697000FBF7CAFE08216846FAF75CFA40B108E066
:1069800026706670D2E72570DAE70BA1FFF77AF878
:10699000A570FEF76BFF0028FBD17CBD0000002036
:1069A000480100204B6579626F6172642073656EE7
:1069B00074204F4B000000004B6579626F61726478
:1069C0002073656E74204641494C45440000000028
:1069D00008B5FAF70FFB00281ED06846FCF710F840
:1069E000002819D00220FCF7DBFF0028FAD004228F
:1069F00069460220FCF74CFE08490322002808885B
:106A000002EB004001D006A100E009A1FFF73AF82F
:106A1000FEF72CFF0028FBD108BD00004801002034
:106A20004D6F7573652073656E74204F4B000000C9
:106A30004D6F7573652073656E74204641494C45F2
:106A40004400000070B5054688690C4600284FF4E4
:106A5000847128460AD0FFF738FCD5F81805626A19
:106A6000E1688854606A401C606270BDFFF72DFCCD
:106A7000D5F8180570BD1FB501238DF80030CDE99C
:106A80000121D0E90012684690471FBD1FB50123C0
:106A90008DF800308DF808100192D0E90012684698
:106AA00090471FBD70B50D4C0020D2B22070201D44
:106AB0000B4D0378EB5C1BB1001DFFF7B3FD02E04B
:106AC0000C30FFF7B5FC08B1F9F71EFF607800281D
:106AD00002D021780029FAD070BD000034000020D7
:106AE000080000202DE9F84F204D924689460646C1
:106AF0009846012269461846AF68F9F7F9FF58B37E
:106B0000009800210446801C09E000BF00EA07034A
:106B10005AF8212005EB8303401C491CDA604145EB
:106B2000F4D34FEA164AFAF741F84AEA0041601CEA
:106B3000384005EB80003C4005EB8402C160D06822
:106B400066F3C50068F3891069F39F2020F0030005
:106B5000401C20F00400D06095F8200402E000BF43
:106B6000FEF784FE0028FBD1BDE8F88FD802002094
:106B700070B50C4605464FF48E71FFF7A6FB216AEF
:106B8000A068415C206A401C2062C5F81C1570BDDD
:106B90001FB500228DF800200291816801914261A9
:106BA000D0E90012684690471FBD00001FB50A4695
:106BB00001788DF8001041680191017A8DF8081074
:106BC000C0680390044850F82210083850F822207A
:106BD000684690471FBD00001400002001490120B5
:106BE000087070473400002010B588B00446202299
:106BF0000E496846F9F796FB06200090C01F0190E9
:106C0000029003904FF0EB7006900CB1084A00E040
:106C1000002269460748FCF7F1F808B1F9F774FE5D
:106C20000448001F447008B010BD0000646F0000ED
:106C3000DD6B0000380000202DE9FF470C460546BB
:106C40004FF40071FFF747FB01274FF4017800264E
:106C500018B34FF4927949462846FFF731FBE0B16B
:106C600049462846FFF731FBC5F8088394F8290008
:106C700000B96F6002208DF80000D5F88004C5F8D7
:106C800080040390A0690290E0680190A661E6612B
:106C9000D4E900126846904728E004212846FFF70F
:106CA0001AFB18B34FF484712846FFF709FBE8B1CB
:106CB00021462846FFF7C6FE616AA069884215D1C1
:106CC000E06938B1E268616AA0612069E6616662E4
:106CD000E06008E094F8290000B96F60C5F8088307
:106CE000A661E268616A2046FFF7C5FE4FF48E7820
:106CF00041462846FFF7E4FA78B1206A6169884284
:106D000002D294F8280020B341462846FFF7DDFA66
:106D1000616911B12046FFF73BFF4FF4A27841466D
:106D20002846FFF7CDFA002818D041462846FFF73D
:106D3000CCFA94F8290000B12F60A06900280DD08A
:106D4000A661E268616A04B02046BDE8F047FFF73B
:106D500092BE21462846FFF70BFFDEE7BDE8FF871E
:106D60001FB50A4601788DF8001041680191017A3B
:106D70008DF80810C0680390044850F822100838B5
:106D800050F82220684690471FBD000014000020E4
:106D90002DE9FF410C464FF4927705463946FFF73F
:106DA000A0FA0026C0B139462846FFF79FFA022014
:106DB0008DF80000D5F88004C5F880040390D5F85C
:106DC0003C058DF80800E0680190A661E661D4E911
:106DD00000126846904723E04FF4887739462846EA
:106DE000FFF77FFAE0B139462846FFF77FFAD5F87A
:106DF0003C15A069884213D1E06960B1E268D5F81A
:106E0000000220F02000C5F80002E069A0612069BE
:106E1000E661E06001E0A661E2682046FFF736FE29
:106E20004FF4A27739462846FFF75BFA60B139463E
:106E30002846FFF75BFAA06930B1A661D5F83C158A
:106E40002046E268FFF722FE4FF490773946284645
:106E5000FFF747FA002813D039462846FFF746FACD
:106E6000606900280CD0D5F84C058DF800608DF8CD
:106E70000800A06801906661D4E900126846904756
:106E8000BDE8FF812DE9F05F8346DDE90A4A9946B6
:106E900090460D460846012703E000BFB0FBF8F01E
:106EA0007F1C4045FAD2B94500D94F465FEACA7007
:106EB00012D18CB15FEA8A7002D5B9F1000F01D00E
:106EC000202607E0302605E031465846641EF9F7D3
:106ED00053FE0CB1A742F7D35FF00106B9F1010FE1
:106EE00002D9A9F1010903E0B5FBF6F0404502D350
:106EF00006FB08F6F2E7DFF83C9000BFB5FBF6F0C2
:106F000000FB165519F800105846F9F735FEB6FB88
:106F1000F8F6002EF2D15FEACA7009D0002C07D033
:106F2000A74205D220215846641EF9F725FEF5E751
:106F3000BDE8F09F486F00000D0E0F100B0C1819E4
:106F40004D630000A96500003031323334353637E7
:106F5000383941424344454609580000DD57000096
:106F6000D5570000FFFFFFFFFFFFFFFFFFFFFFFF01
:106F7000FFFFFFFF00000000000000000000D6013E
:106F80000701000032536601172D2D1A440C4023CF
:106F9000490D171A2D0B4D000000000000000000E5
:106FA0000338FDD870470000001000401011004069
:106FB000031000000100000000100040000000006D
:106FC0000B0204000000000004100040000000005C
:106FD00007010301000000000040404040404040E5
:106FE000404041414141414040404040404040409C
:106FF0004040404040404040400502020202020240
:10700000020202020202020202202020202020208E
:1070100020202002020202020202909090909090A2
:107020001010101010101010101010101010101060
:1070300010101010020202020202888888888888D4
:1070400008080808080808080808080808080808C0
:10705000080808080202020240000000D96F000080
:107060007761726E696E6700646562756700000023
:107070001B5B313B33306D001B5B306D000000004B
:107080001B5B313B33316D001B5B313B33326D0099
:107090001B5B313B33336D001B5B313B33346D0085
:1070A0001B5B313B33356D001B5B313B33366D0071
:1070B0001B5B313B33376D00696E666F000000006B
:1070C0006572726F72000000505253005541525465
:1070D00000000000554152544500000062616C6C94
:1070E0006F632E6C6F675F6D656D706F6F6C000006
:1070F0006170700054710000000000204C0100001D
:10710000B8030000A47100004C010020B419000075
:107110007C080000C870000000000000CC70000077
:1071200000000000D470000000000000DC700000CF
:1071300000000003F0700000000003036000002066
:1071400058000020600000201802002044010020A8
:10715000180000004104380101016420004054205F
:1071600000400327586F33C07033607033B87033FA
:1071700068703378703370703380703388703390F8
:107180007033987033A07033A8700320B07004116E
:1071900090D003C205064404192A3F4D33414803E9
:0471A0001B05480083
:0400000500000201F4
:00000001FF
